******************************************************************************
             TMS320C2000 Linker PC v16.9.6                     
******************************************************************************
>> Linked Wed Jan 17 02:13:41 2018

OUTPUT FILE NAME:   <usb_dev_serial.out>
ENTRY POINT SYMBOL: "_c_int00"  address: 0000d3ab


MEMORY CONFIGURATION

         name            origin    length      used     unused   attr    fill
----------------------  --------  ---------  --------  --------  ----  --------
PAGE 0:
  BEGIN                 00000000   00000002  00000002  00000000  RWIX
  RAMM0                 00000050   000003b0  0000010e  000002a2  RWIX
  RAML0_L5              00008000   00006000  000055a6  00000a5a  RWIX
  FPUTABLES             003fd860   000006a0  00000000  000006a0  RWIX
  IQTABLES              003fdf00   00000b50  00000000  00000b50  RWIX
  IQTABLES2             003fea50   0000008c  00000000  0000008c  RWIX
  IQTABLES3             003feadc   000000aa  00000000  000000aa  RWIX
  BOOTROM               003ff3b0   00000c10  00000000  00000c10  RWIX
  RESET                 003fffc0   00000002  00000000  00000002  RWIX

PAGE 1:
  BOOT_RSVD             00000002   0000004e  00000000  0000004e  RWIX
  RAMM1                 00000400   00000400  00000400  00000000  RWIX
  DEV_EMU               00000880   00000105  00000004  00000101  RWIX
  SYS_PWR_CTL           00000985   00000003  00000003  00000000  RWIX
  FLASH_REGS            00000a80   00000060  00000008  00000058  RWIX
  CSM                   00000ae0   00000020  00000010  00000010  RWIX
  ADC_RESULT            00000b00   00000020  00000010  00000010  RWIX
  CPU_TIMER0            00000c00   00000008  00000008  00000000  RWIX
  CPU_TIMER1            00000c08   00000008  00000008  00000000  RWIX
  CPU_TIMER2            00000c10   00000008  00000008  00000000  RWIX
  PIE_CTRL              00000ce0   00000020  0000001a  00000006  RWIX
  PIE_VECT              00000d00   00000100  00000100  00000000  RWIX
  DMA                   00001000   00000200  000000e0  00000120  RWIX
  CLA1                  00001400   00000080  00000040  00000040  RWIX
  USB0                  00004000   00001000  00000454  00000bac  RWIX
  McBSPA                00005000   00000040  00000024  0000001c  RWIX
  ECANA                 00006000   00000040  00000034  0000000c  RWIX
  ECANA_LAM             00006040   00000040  00000040  00000000  RWIX
  ECANA_MOTS            00006080   00000040  00000040  00000000  RWIX
  ECANA_MOTO            000060c0   00000040  00000040  00000000  RWIX
  ECANA_MBOX            00006100   00000100  00000100  00000000  RWIX
  COMP1                 00006400   00000020  00000014  0000000c  RWIX
  COMP2                 00006420   00000020  00000014  0000000c  RWIX
  COMP3                 00006440   00000020  00000014  0000000c  RWIX
  EPWM1                 00006800   00000040  00000040  00000000  RWIX
  EPWM2                 00006840   00000040  00000040  00000000  RWIX
  EPWM3                 00006880   00000040  00000040  00000000  RWIX
  EPWM4                 000068c0   00000040  00000040  00000000  RWIX
  EPWM5                 00006900   00000040  00000040  00000000  RWIX
  EPWM6                 00006940   00000040  00000040  00000000  RWIX
  EPWM7                 00006980   00000040  00000040  00000000  RWIX
  EPWM8                 000069c0   00000040  00000040  00000000  RWIX
  ECAP1                 00006a00   00000020  00000020  00000000  RWIX
  ECAP2                 00006a20   00000020  00000020  00000000  RWIX
  ECAP3                 00006a40   00000020  00000020  00000000  RWIX
  HRCAP1                00006ac0   00000020  00000020  00000000  RWIX
  HRCAP2                00006ae0   00000020  00000020  00000000  RWIX
  EQEP1                 00006b00   00000040  00000022  0000001e  RWIX
  EQEP2                 00006b40   00000040  00000022  0000001e  RWIX
  HRCAP3                00006c80   00000020  00000020  00000000  RWIX
  HRCAP4                00006ca0   00000020  00000020  00000000  RWIX
  GPIOCTRL              00006f80   00000040  00000040  00000000  RWIX
  GPIODAT               00006fc0   00000020  00000020  00000000  RWIX
  GPIOINT               00006fe0   00000020  00000020  00000000  RWIX
  SYSTEM                00007010   00000030  00000030  00000000  RWIX
  SPIA                  00007040   00000010  00000010  00000000  RWIX
  SCIA                  00007050   00000010  00000010  00000000  RWIX
  NMIINTRUPT            00007060   00000010  00000010  00000000  RWIX
  XINTRUPT              00007070   00000010  00000010  00000000  RWIX
  ADC                   00007100   00000080  00000050  00000030  RWIX
  SPIB                  00007740   00000010  00000010  00000000  RWIX
  SCIB                  00007750   00000010  00000010  00000000  RWIX
  I2CA                  00007900   00000040  00000022  0000001e  RWIX
  RAML6                 0000e000   00002000  00000ad8  00001528  RWIX
  RAML7                 00010000   00002000  00000000  00002000  RWIX
  RAML8                 00012000   00002000  00000000  00002000  RWIX
  USB_RAM               00040000   00000800  00000000  00000800  RWIX
  PARTID                003d7e80   00000001  00000001  00000000  RWIX
  CSM_PWL               003f7ff8   00000008  00000008  00000000  RWIX


SECTION ALLOCATION MAP

 output                                  attributes/
section   page    origin      length       input sections
--------  ----  ----------  ----------   ----------------
codestart 
*          0    00000000    00000002     
                  00000000    00000002     F2806x_CodeStartBranch_ebss_init.obj (codestart)

.cinit     0    00000050    000000e4     
                  00000050    00000046     usblib.lib : usbhostenum.obj (.cinit)
                  00000096    00000040                : usbdcdc.obj (.cinit)
                  000000d6    00000017     usb_serial_structs.obj (.cinit)
                  000000ed    0000000e     rts2800_fpu32.lib : exit.obj (.cinit)
                  000000fb    0000000e     usblib.lib : usbtick.obj (.cinit)
                  00000109    0000000d                : usbmode.obj (.cinit)
                  00000116    00000009     uartstdio.obj (.cinit)
                  0000011f    00000005     rts2800_fpu32.lib : _lock.obj (.cinit:__lock)
                  00000124    00000005                       : _lock.obj (.cinit:__unlock)
                  00000129    00000005     usblib.lib : usbdenum.obj (.cinit)
                  0000012e    00000004     usb_dev_serial.obj (.cinit)
                  00000132    00000002     --HOLE-- [fill = 0]

.switch    0    00000134    0000002a     
                  00000134    0000002a     usblib.lib : usbdcdc.obj (.switch:_HandleRequests)

.text      0    00008000    000055a6     
                  00008000    000015cf     usblib.lib : usbhostenum.obj (.text)
                  000095cf    00000e95     usb.obj (.text)
                  0000a464    0000083e     usblib.lib : usbdenum.obj (.text)
                  0000aca2    00000728                : usbdcdc.obj (.text)
                  0000b3ca    000003fe                : usbhhub.obj (.text)
                  0000b7c8    0000039b     F2806x_DefaultIsr.obj (.text:retain)
                  0000bb63    000002ae     uartstdio.obj (.text)
                  0000be11    00000291     usb_dev_serial.obj (.text)
                  0000c0a2    0000028f     driverlib.lib : uart.obj (.text)
                  0000c331    00000257     usblib.lib : usbbuffer.obj (.text)
                  0000c588    00000255                : usbmode.obj (.text)
                  0000c7dd    000001fd                : usbdconfig.obj (.text)
                  0000c9da    0000019d     driverlib.lib : interrupt.obj (.text)
                  0000cb77    00000150     usblib.lib : usbdcdesc.obj (.text)
                  0000ccc7    00000146                : usbringbuf.obj (.text)
                  0000ce0d    000000d2                : usbdma.obj (.text)
                  0000cedf    000000cb                : usbdesc.obj (.text)
                  0000cfaa    000000ac     sysctl.obj (.text)
                  0000d056    0000009c     rts2800_fpu32.lib : fd_add28.obj (.text)
                  0000d0f2    00000096     usb_dev_serial.obj (.text:retain)
                  0000d188    00000093     usb_hal.obj (.text:retain)
                  0000d21b    0000008b     rts2800_fpu32.lib : fd_div28.obj (.text)
                  0000d2a6    00000083                       : fd_mpy28.obj (.text)
                  0000d329    00000082     usblib.lib : usbtick.obj (.text)
                  0000d3ab    00000056     rts2800_fpu32.lib : boot28.obj (.text)
                  0000d401    00000052     usb_hal.obj (.text)
                  0000d453    00000029     rts2800_fpu32.lib : exit.obj (.text)
                  0000d47c    00000028     F2806x_PieCtrl.obj (.text)
                  0000d4a4    00000026     F2806x_PieVect.obj (.text)
                  0000d4ca    00000024     rts2800_fpu32.lib : cpy_tbl.obj (.text)
                  0000d4ee    0000001e                       : memcpy.obj (.text)
                  0000d50c    0000001b                       : fd_toul28.obj (.text)
                  0000d527    00000019                       : args_main.obj (.text)
                  0000d540    00000016                       : ul_tofd28.obj (.text)
                  0000d556    00000013     F2806x_CodeStartBranch_ebss_init.obj (.text)
                  0000d569    00000012     usblib.lib : usbdhandler.obj (.text)
                  0000d57b    0000000e     rts2800_fpu32.lib : fd_sub28.obj (.text)
                  0000d589    0000000d     driverlib.lib : interrupt.obj (.text:retain)
                  0000d596    00000009     rts2800_fpu32.lib : _lock.obj (.text)
                  0000d59f    00000004     F2806x_usDelay.obj (.text)
                  0000d5a3    00000002     rts2800_fpu32.lib : pre_init.obj (.text)
                  0000d5a5    00000001                       : startup.obj (.text)

.pinit     0    00000050    00000000     UNINITIALIZED

.reset     0    003fffc0    00000002     DSECT
                  003fffc0    00000002     rts2800_fpu32.lib : boot28.obj (.reset)

.stack     1    00000400    00000400     UNINITIALIZED
                  00000400    00000400     --HOLE--

DevEmuRegsFile 
*          1    00000880    00000004     UNINITIALIZED
                  00000880    00000004     F2806x_GlobalVariableDefs.obj (DevEmuRegsFile)

SysPwrCtrlRegsFile 
*          1    00000985    00000003     UNINITIALIZED
                  00000985    00000003     F2806x_GlobalVariableDefs.obj (SysPwrCtrlRegsFile)

FlashRegsFile 
*          1    00000a80    00000008     UNINITIALIZED
                  00000a80    00000008     F2806x_GlobalVariableDefs.obj (FlashRegsFile)

CsmRegsFile 
*          1    00000ae0    00000010     UNINITIALIZED
                  00000ae0    00000010     F2806x_GlobalVariableDefs.obj (CsmRegsFile)

AdcResultFile 
*          1    00000b00    00000010     UNINITIALIZED
                  00000b00    00000010     F2806x_GlobalVariableDefs.obj (AdcResultFile)

CpuTimer0RegsFile 
*          1    00000c00    00000008     UNINITIALIZED
                  00000c00    00000008     F2806x_GlobalVariableDefs.obj (CpuTimer0RegsFile)

CpuTimer1RegsFile 
*          1    00000c08    00000008     UNINITIALIZED
                  00000c08    00000008     F2806x_GlobalVariableDefs.obj (CpuTimer1RegsFile)

CpuTimer2RegsFile 
*          1    00000c10    00000008     UNINITIALIZED
                  00000c10    00000008     F2806x_GlobalVariableDefs.obj (CpuTimer2RegsFile)

PieCtrlRegsFile 
*          1    00000ce0    0000001a     UNINITIALIZED
                  00000ce0    0000001a     F2806x_GlobalVariableDefs.obj (PieCtrlRegsFile)

PieVectTableFile 
*          1    00000d00    00000100     UNINITIALIZED
                  00000d00    00000100     F2806x_GlobalVariableDefs.obj (PieVectTableFile)

EmuKeyVar 
*          1    00000d00    00000001     UNINITIALIZED
                  00000d00    00000001     F2806x_GlobalVariableDefs.obj (EmuKeyVar)

EmuBModeVar 
*          1    00000d01    00000001     UNINITIALIZED
                  00000d01    00000001     F2806x_GlobalVariableDefs.obj (EmuBModeVar)

FlashCallbackVar 
*          1    00000d02    00000002     UNINITIALIZED
                  00000d02    00000002     F2806x_GlobalVariableDefs.obj (FlashCallbackVar)

FlashScalingVar 
*          1    00000d04    00000002     UNINITIALIZED
                  00000d04    00000002     F2806x_GlobalVariableDefs.obj (FlashScalingVar)

DmaRegsFile 
*          1    00001000    000000e0     UNINITIALIZED
                  00001000    000000e0     F2806x_GlobalVariableDefs.obj (DmaRegsFile)

Cla1RegsFile 
*          1    00001400    00000040     UNINITIALIZED
                  00001400    00000040     F2806x_GlobalVariableDefs.obj (Cla1RegsFile)

Usb0RegsFile 
*          1    00004000    00000454     UNINITIALIZED
                  00004000    00000454     F2806x_GlobalVariableDefs.obj (Usb0RegsFile)

McbspaRegsFile 
*          1    00005000    00000024     UNINITIALIZED
                  00005000    00000024     F2806x_GlobalVariableDefs.obj (McbspaRegsFile)

ECanaRegsFile 
*          1    00006000    00000034     UNINITIALIZED
                  00006000    00000034     F2806x_GlobalVariableDefs.obj (ECanaRegsFile)

ECanaLAMRegsFile 
*          1    00006040    00000040     UNINITIALIZED
                  00006040    00000040     F2806x_GlobalVariableDefs.obj (ECanaLAMRegsFile)

ECanaMOTSRegsFile 
*          1    00006080    00000040     UNINITIALIZED
                  00006080    00000040     F2806x_GlobalVariableDefs.obj (ECanaMOTSRegsFile)

ECanaMOTORegsFile 
*          1    000060c0    00000040     UNINITIALIZED
                  000060c0    00000040     F2806x_GlobalVariableDefs.obj (ECanaMOTORegsFile)

ECanaMboxesFile 
*          1    00006100    00000100     UNINITIALIZED
                  00006100    00000100     F2806x_GlobalVariableDefs.obj (ECanaMboxesFile)

Comp1RegsFile 
*          1    00006400    00000014     UNINITIALIZED
                  00006400    00000014     F2806x_GlobalVariableDefs.obj (Comp1RegsFile)

Comp2RegsFile 
*          1    00006420    00000014     UNINITIALIZED
                  00006420    00000014     F2806x_GlobalVariableDefs.obj (Comp2RegsFile)

Comp3RegsFile 
*          1    00006440    00000014     UNINITIALIZED
                  00006440    00000014     F2806x_GlobalVariableDefs.obj (Comp3RegsFile)

EPwm1RegsFile 
*          1    00006800    00000040     UNINITIALIZED
                  00006800    00000040     F2806x_GlobalVariableDefs.obj (EPwm1RegsFile)

EPwm2RegsFile 
*          1    00006840    00000040     UNINITIALIZED
                  00006840    00000040     F2806x_GlobalVariableDefs.obj (EPwm2RegsFile)

EPwm3RegsFile 
*          1    00006880    00000040     UNINITIALIZED
                  00006880    00000040     F2806x_GlobalVariableDefs.obj (EPwm3RegsFile)

EPwm4RegsFile 
*          1    000068c0    00000040     UNINITIALIZED
                  000068c0    00000040     F2806x_GlobalVariableDefs.obj (EPwm4RegsFile)

EPwm5RegsFile 
*          1    00006900    00000040     UNINITIALIZED
                  00006900    00000040     F2806x_GlobalVariableDefs.obj (EPwm5RegsFile)

EPwm6RegsFile 
*          1    00006940    00000040     UNINITIALIZED
                  00006940    00000040     F2806x_GlobalVariableDefs.obj (EPwm6RegsFile)

EPwm7RegsFile 
*          1    00006980    00000040     UNINITIALIZED
                  00006980    00000040     F2806x_GlobalVariableDefs.obj (EPwm7RegsFile)

EPwm8RegsFile 
*          1    000069c0    00000040     UNINITIALIZED
                  000069c0    00000040     F2806x_GlobalVariableDefs.obj (EPwm8RegsFile)

ECap1RegsFile 
*          1    00006a00    00000020     UNINITIALIZED
                  00006a00    00000020     F2806x_GlobalVariableDefs.obj (ECap1RegsFile)

ECap2RegsFile 
*          1    00006a20    00000020     UNINITIALIZED
                  00006a20    00000020     F2806x_GlobalVariableDefs.obj (ECap2RegsFile)

ECap3RegsFile 
*          1    00006a40    00000020     UNINITIALIZED
                  00006a40    00000020     F2806x_GlobalVariableDefs.obj (ECap3RegsFile)

HRCap1RegsFile 
*          1    00006ac0    00000020     UNINITIALIZED
                  00006ac0    00000020     F2806x_GlobalVariableDefs.obj (HRCap1RegsFile)

HRCap2RegsFile 
*          1    00006ae0    00000020     UNINITIALIZED
                  00006ae0    00000020     F2806x_GlobalVariableDefs.obj (HRCap2RegsFile)

EQep1RegsFile 
*          1    00006b00    00000022     UNINITIALIZED
                  00006b00    00000022     F2806x_GlobalVariableDefs.obj (EQep1RegsFile)

EQep2RegsFile 
*          1    00006b40    00000022     UNINITIALIZED
                  00006b40    00000022     F2806x_GlobalVariableDefs.obj (EQep2RegsFile)

HRCap3RegsFile 
*          1    00006c80    00000020     UNINITIALIZED
                  00006c80    00000020     F2806x_GlobalVariableDefs.obj (HRCap3RegsFile)

HRCap4RegsFile 
*          1    00006ca0    00000020     UNINITIALIZED
                  00006ca0    00000020     F2806x_GlobalVariableDefs.obj (HRCap4RegsFile)

GpioCtrlRegsFile 
*          1    00006f80    00000040     UNINITIALIZED
                  00006f80    00000040     F2806x_GlobalVariableDefs.obj (GpioCtrlRegsFile)

GpioDataRegsFile 
*          1    00006fc0    00000020     UNINITIALIZED
                  00006fc0    00000020     F2806x_GlobalVariableDefs.obj (GpioDataRegsFile)

GpioIntRegsFile 
*          1    00006fe0    00000020     UNINITIALIZED
                  00006fe0    00000020     F2806x_GlobalVariableDefs.obj (GpioIntRegsFile)

SysCtrlRegsFile 
*          1    00007010    00000030     UNINITIALIZED
                  00007010    00000030     F2806x_GlobalVariableDefs.obj (SysCtrlRegsFile)

SpiaRegsFile 
*          1    00007040    00000010     UNINITIALIZED
                  00007040    00000010     F2806x_GlobalVariableDefs.obj (SpiaRegsFile)

SciaRegsFile 
*          1    00007050    00000010     UNINITIALIZED
                  00007050    00000010     F2806x_GlobalVariableDefs.obj (SciaRegsFile)

NmiIntruptRegsFile 
*          1    00007060    00000010     UNINITIALIZED
                  00007060    00000010     F2806x_GlobalVariableDefs.obj (NmiIntruptRegsFile)

XIntruptRegsFile 
*          1    00007070    00000010     UNINITIALIZED
                  00007070    00000010     F2806x_GlobalVariableDefs.obj (XIntruptRegsFile)

AdcRegsFile 
*          1    00007100    00000050     UNINITIALIZED
                  00007100    00000050     F2806x_GlobalVariableDefs.obj (AdcRegsFile)

SpibRegsFile 
*          1    00007740    00000010     UNINITIALIZED
                  00007740    00000010     F2806x_GlobalVariableDefs.obj (SpibRegsFile)

ScibRegsFile 
*          1    00007750    00000010     UNINITIALIZED
                  00007750    00000010     F2806x_GlobalVariableDefs.obj (ScibRegsFile)

I2caRegsFile 
*          1    00007900    00000022     UNINITIALIZED
                  00007900    00000022     F2806x_GlobalVariableDefs.obj (I2caRegsFile)

.ebss      1    0000e000    000007c0     
                  0000e000    0000038e     usblib.lib : usbhostenum.obj (.ebss) [fill = 0000]
                  0000e38e    00000031                : usbdcdc.obj (.ebss) [fill = 0000]
                  0000e3bf    00000001     usb_dev_serial.obj (.ebss) [fill = 0000]
                  0000e3c0    00000280     usb_serial_structs.obj (.ebss) [fill = 0000]
                  0000e640    0000008c     usblib.lib : usbdma.obj (.ebss) [fill = 0000]
                  0000e6cc    0000001e                : usbtick.obj (.ebss) [fill = 0000]
                  0000e6ea    0000000a                : usbmode.obj (.ebss) [fill = 0000]
                  0000e6f4    00000006     rts2800_fpu32.lib : exit.obj (.ebss) [fill = 0000]
                  0000e6fa    00000004     uartstdio.obj (.ebss) [fill = 0000]
                  0000e6fe    00000002     rts2800_fpu32.lib : _lock.obj (.ebss:__lock) [fill = 0000]
                  0000e700    00000080     usblib.lib : usbdenum.obj (.ebss) [fill = 0000]
                  0000e780    0000003e                : usbhhub.obj (.ebss) [fill = 0000]
                  0000e7be    00000002     rts2800_fpu32.lib : _lock.obj (.ebss:__unlock) [fill = 0000]

.econst    1    0000e7c0    00000318     
                  0000e7c0    00000100     F2806x_PieVect.obj (.econst:_PieVectTableInit)
                  0000e8c0    0000004d     usb.obj (.econst:.string)
                  0000e90d    00000036     usb_serial_structs.obj (.econst:_g_pui8ConfigString)
                  0000e943    00000001     --HOLE-- [fill = 0]
                  0000e944    00000032     uartstdio.obj (.econst:.string)
                  0000e976    0000002c     usb_serial_structs.obj (.econst:_g_pui8ControlInterfaceString)
                  0000e9a2    00000024     usb_serial_structs.obj (.econst:_g_pui8ManufacturerString)
                  0000e9c6    00000023     usblib.lib : usbdcdc.obj (.econst:_g_pui8CDCSerCommInterface)
                  0000e9e9    00000022     usb_serial_structs.obj (.econst:_g_pui8ProdectString)
                  0000ea0b    00000001     --HOLE-- [fill = 0]
                  0000ea0c    0000001a     usblib.lib : usbdenum.obj (.econst:_g_psUSBDStdRequests)
                  0000ea26    00000018                : usbdcdc.obj (.econst:_g_sCDCHandlers)
                  0000ea3e    00000017                : usbdcdc.obj (.econst:_g_pui8CDCSerDataInterface)
                  0000ea55    00000012     usb_serial_structs.obj (.econst:_g_pui8SerialNumberString)
                  0000ea67    00000001     --HOLE-- [fill = 0]
                  0000ea68    00000012     usb_serial_structs.obj (.econst:_g_sRxBuffer)
                  0000ea7a    00000012     usb_serial_structs.obj (.econst:_g_sTxBuffer)
                  0000ea8c    00000010     usb_hal.obj (.econst)
                  0000ea9c    0000000c     usb_serial_structs.obj (.econst:_g_pui8StringDescriptors)
                  0000eaa8    00000006     uartstdio.obj (.econst:_g_ulUARTBase)
                  0000eaae    00000006     uartstdio.obj (.econst:_g_ulUARTPeriph)
                  0000eab4    00000004     usb_serial_structs.obj (.econst:_g_pui8LangDescriptor)
                  0000eab8    00000004     usblib.lib : usbdcdc.obj (.econst:_g_sCDCCompSerConfigHeader)
                  0000eabc    00000004                : usbdcdc.obj (.econst:_g_sCDCSerCommInterfaceSection)
                  0000eac0    00000004                : usbdcdc.obj (.econst:_g_sCDCSerConfigHeader)
                  0000eac4    00000004                : usbdcdc.obj (.econst:_g_sCDCSerConfigSection)
                  0000eac8    00000004                : usbdcdc.obj (.econst:_g_sCDCSerDataInterfaceSection)
                  0000eacc    00000004                : usbdcdc.obj (.econst:_g_sIADSerConfigSection)
                  0000ead0    00000002     usb_dev_serial.obj (.econst:.string)
                  0000ead2    00000002     usblib.lib : usbdcdc.obj (.econst:_g_pCDCCompSerConfigDescriptors)
                  0000ead4    00000002                : usbdcdc.obj (.econst:_g_ppCDCSerConfigDescriptors)
                  0000ead6    00000002     uartstdio.obj (.econst)

PartIdRegsFile 
*          1    003d7e80    00000001     UNINITIALIZED
                  003d7e80    00000001     F2806x_GlobalVariableDefs.obj (PartIdRegsFile)

CsmPwlFile 
*          1    003f7ff8    00000008     UNINITIALIZED
                  003f7ff8    00000008     F2806x_GlobalVariableDefs.obj (CsmPwlFile)

MODULE SUMMARY

       Module                                 code    initialized data   uninitialized data
       ------                                 ----    ----------------   ------------------
    .\
       usb.obj                                3733    77                 0                 
       F2806x_GlobalVariableDefs.obj          0       0                  3550              
       F2806x_DefaultIsr.obj                  923     0                  0                 
       usb_serial_structs.obj                 0       901                0                 
       usb_dev_serial.obj                     807     7                  0                 
       uartstdio.obj                          686     77                 0                 
       F2806x_PieVect.obj                     38      256                0                 
       usb_hal.obj                            229     16                 0                 
       sysctl.obj                             172     0                  0                 
       F2806x_PieCtrl.obj                     40      0                  0                 
       F2806x_CodeStartBranch_ebss_init.obj   21      0                  0                 
       F2806x_usDelay.obj                     4       0                  0                 
    +--+--------------------------------------+-------+------------------+--------------------+
       Total:                                 6653    1334               3550              
                                                                                           
    F:/ti/c2000/C2000Ware_1_00_03_00/device_support/f2806x/MWare/driverlib/Debug/driverlib.lib
       uart.obj                               655     0                  0                 
       interrupt.obj                          426     0                  0                 
    +--+--------------------------------------+-------+------------------+--------------------+
       Total:                                 1081    0                  0                 
                                                                                           
    F:/ti/c2000/C2000Ware_1_00_03_00/libraries/communications/usb/f2806x/lib/usblib.lib
       usbhostenum.obj                        5583    980                0                 
       usbdenum.obj                           2110    159                0                 
       usbdcdc.obj                            1832    265                0                 
       usbhhub.obj                            1022    62                 0                 
       usbmode.obj                            597     23                 0                 
       usbbuffer.obj                          599     0                  0                 
       usbdconfig.obj                         509     0                  0                 
       usbdma.obj                             210     140                0                 
       usbdcdesc.obj                          336     0                  0                 
       usbringbuf.obj                         326     0                  0                 
       usbdesc.obj                            203     0                  0                 
       usbtick.obj                            130     44                 0                 
       usbdhandler.obj                        18      0                  0                 
    +--+--------------------------------------+-------+------------------+--------------------+
       Total:                                 13475   1673               0                 
                                                                                           
    F:\TI_CCS_7P4\ccsv7\tools\compiler\ti-cgt-c2000_16.9.6.LTS\lib\rts2800_fpu32.lib
       fd_add28.obj                           156     0                  0                 
       fd_div28.obj                           139     0                  0                 
       fd_mpy28.obj                           131     0                  0                 
       boot28.obj                             86      0                  0                 
       exit.obj                               41      20                 0                 
       cpy_tbl.obj                            36      0                  0                 
       memcpy.obj                             30      0                  0                 
       fd_toul28.obj                          27      0                  0                 
       args_main.obj                          25      0                  0                 
       _lock.obj                              9       14                 0                 
       ul_tofd28.obj                          22      0                  0                 
       fd_sub28.obj                           14      0                  0                 
       pre_init.obj                           2       0                  0                 
       startup.obj                            1       0                  0                 
    +--+--------------------------------------+-------+------------------+--------------------+
       Total:                                 719     34                 0                 
                                                                                           
       Stack:                                 0       0                  1024              
    +--+--------------------------------------+-------+------------------+--------------------+
       Grand Total:                           21928   3041               4574              


GLOBAL DATA SYMBOLS: SORTED BY DATA PAGE

address     data page           name
--------    ----------------    ----
00000400      10 (00000400)     __stack

00000880      22 (00000880)     _DevEmuRegs

00000985      26 (00000980)     _SysPwrCtrlRegs

00000a80      2a (00000a80)     _FlashRegs

00000ae0      2b (00000ac0)     _CsmRegs

00000b00      2c (00000b00)     _AdcResult

00000c00      30 (00000c00)     _CpuTimer0Regs
00000c08      30 (00000c00)     _CpuTimer1Regs
00000c10      30 (00000c00)     _CpuTimer2Regs

00000ce0      33 (00000cc0)     _PieCtrlRegs

00000d00      34 (00000d00)     _EmuKey
00000d00      34 (00000d00)     _PieVectTable
00000d01      34 (00000d00)     _EmuBMode
00000d02      34 (00000d00)     _Flash_CallbackPtr
00000d04      34 (00000d00)     _Flash_CPUScaleFactor

00001000      40 (00001000)     _DmaRegs

00001400      50 (00001400)     _Cla1Regs

00004000     100 (00004000)     _Usb0Regs

00005000     140 (00005000)     _McbspaRegs

00006000     180 (00006000)     _ECanaRegs

00006040     181 (00006040)     _ECanaLAMRegs

00006080     182 (00006080)     _ECanaMOTSRegs

000060c0     183 (000060c0)     _ECanaMOTORegs

00006100     184 (00006100)     _ECanaMboxes

00006400     190 (00006400)     _Comp1Regs
00006420     190 (00006400)     _Comp2Regs

00006440     191 (00006440)     _Comp3Regs

00006800     1a0 (00006800)     _EPwm1Regs

00006840     1a1 (00006840)     _EPwm2Regs

00006880     1a2 (00006880)     _EPwm3Regs

000068c0     1a3 (000068c0)     _EPwm4Regs

00006900     1a4 (00006900)     _EPwm5Regs

00006940     1a5 (00006940)     _EPwm6Regs

00006980     1a6 (00006980)     _EPwm7Regs

000069c0     1a7 (000069c0)     _EPwm8Regs

00006a00     1a8 (00006a00)     _ECap1Regs
00006a20     1a8 (00006a00)     _ECap2Regs

00006a40     1a9 (00006a40)     _ECap3Regs

00006ac0     1ab (00006ac0)     _HRCap1Regs
00006ae0     1ab (00006ac0)     _HRCap2Regs

00006b00     1ac (00006b00)     _EQep1Regs

00006b40     1ad (00006b40)     _EQep2Regs

00006c80     1b2 (00006c80)     _HRCap3Regs
00006ca0     1b2 (00006c80)     _HRCap4Regs

00006f80     1be (00006f80)     _GpioCtrlRegs

00006fc0     1bf (00006fc0)     _GpioDataRegs
00006fe0     1bf (00006fc0)     _GpioIntRegs

00007010     1c0 (00007000)     _SysCtrlRegs

00007040     1c1 (00007040)     _SpiaRegs
00007050     1c1 (00007040)     _SciaRegs
00007060     1c1 (00007040)     _NmiIntruptRegs
00007070     1c1 (00007040)     _XIntruptRegs

00007100     1c4 (00007100)     _AdcRegs

00007740     1dd (00007740)     _SpibRegs
00007750     1dd (00007740)     _ScibRegs

00007900     1e4 (00007900)     _I2caRegs

0000e38e     38e (0000e380)     _g_psCDCSerSections
0000e394     38e (0000e380)     _g_psCDCCompSerSections
0000e39c     38e (0000e380)     _g_pui8IADSerDescriptor
0000e3a4     38e (0000e380)     _g_pui8CDCSerDescriptor
0000e3ad     38e (0000e380)     _g_pui8CDCSerDeviceDescriptor

0000e3c0     38f (0000e3c0)     _g_pui8TxBufferWorkspace
0000e3d8     38f (0000e3c0)     _g_pui8RxBufferWorkspace

0000e400     390 (0000e400)     _g_sCDCDevice

0000e440     391 (0000e440)     _g_pi8USBRxBuffer

0000e540     395 (0000e540)     _g_pi8USBTxBuffer

0000e6cc     39b (0000e6c0)     _g_bUSBTimerInitialized
0000e6ce     39b (0000e6c0)     _g_ui32CurrentUSBTick
0000e6d0     39b (0000e6c0)     _g_ui32USBSOFCount
0000e6d2     39b (0000e6c0)     _g_pfnTickHandlers
0000e6de     39b (0000e6c0)     _g_pvTickInstance
0000e6eb     39b (0000e6c0)     _g_iUSBMode
0000e6ec     39b (0000e6c0)     _g_eOTGModeState
0000e6f0     39b (0000e6c0)     _g_ui32PollRate
0000e6f2     39b (0000e6c0)     _g_ui32WaitTicks
0000e6f4     39b (0000e6c0)     ___TI_enable_exit_profile_output
0000e6f6     39b (0000e6c0)     ___TI_cleanup_ptr
0000e6f8     39b (0000e6c0)     ___TI_dtors_ptr
0000e6fe     39b (0000e6c0)     __lock

0000e700     39c (0000e700)     _g_ppsDevInfo
0000e704     39c (0000e700)     _g_psDCDInst

0000e7be     39e (0000e780)     __unlock

0000e7c0     39f (0000e7c0)     _PieVectTableInit

0000e90d     3a4 (0000e900)     _g_pui8ConfigString

0000e976     3a5 (0000e940)     _g_pui8ControlInterfaceString

0000e9a2     3a6 (0000e980)     _g_pui8ManufacturerString

0000e9c6     3a7 (0000e9c0)     _g_pui8CDCSerCommInterface
0000e9e9     3a7 (0000e9c0)     _g_pui8ProdectString

0000ea26     3a8 (0000ea00)     _g_sCDCHandlers
0000ea3e     3a8 (0000ea00)     _g_pui8CDCSerDataInterface

0000ea55     3a9 (0000ea40)     _g_pui8SerialNumberString
0000ea68     3a9 (0000ea40)     _g_sRxBuffer
0000ea7a     3a9 (0000ea40)     _g_sTxBuffer

0000ea9c     3aa (0000ea80)     _g_pui8StringDescriptors
0000eab4     3aa (0000ea80)     _g_pui8LangDescriptor
0000eab8     3aa (0000ea80)     _g_sCDCCompSerConfigHeader
0000eabc     3aa (0000ea80)     _g_sCDCSerCommInterfaceSection

0000eac0     3ab (0000eac0)     _g_sCDCSerConfigHeader
0000eac4     3ab (0000eac0)     _g_sCDCSerConfigSection
0000eac8     3ab (0000eac0)     _g_sCDCSerDataInterfaceSection
0000eacc     3ab (0000eac0)     _g_sIADSerConfigSection
0000ead2     3ab (0000eac0)     _g_pCDCCompSerConfigDescriptors
0000ead4     3ab (0000eac0)     _g_ppCDCSerConfigDescriptors

003d7e80    f5fa (003d7e80)     _PartIdRegs

003f7ff8    fdff (003f7fc0)     _CsmPwl


GLOBAL SYMBOLS: SORTED ALPHABETICALLY BY Name 

page  address   name                                  
----  -------   ----                                  
0     00008000  .text                                 
0     0000d453  C$$EXIT                               
0     0000d056  FD$$ADD                               
0     0000d21b  FD$$DIV                               
0     0000d2a6  FD$$MPY                               
0     0000d57b  FD$$SUB                               
0     0000d50c  FD$$TOUL                              
0     0000d540  UL$$TOFD                              
0     0000b886  _ADCINT1_ISR                          
0     0000b890  _ADCINT2_ISR                          
0     0000ba98  _ADCINT3_ISR                          
0     0000baa2  _ADCINT4_ISR                          
0     0000baac  _ADCINT5_ISR                          
0     0000bab6  _ADCINT6_ISR                          
0     0000bac0  _ADCINT7_ISR                          
0     0000baca  _ADCINT8_ISR                          
0     0000b8ae  _ADCINT9_ISR                          
1     00007100  _AdcRegs                              
1     00000b00  _AdcResult                            
0     0000bad4  _CLA1_INT1_ISR                        
0     0000bade  _CLA1_INT2_ISR                        
0     0000bae8  _CLA1_INT3_ISR                        
0     0000baf2  _CLA1_INT4_ISR                        
0     0000bafc  _CLA1_INT5_ISR                        
0     0000bb06  _CLA1_INT6_ISR                        
0     0000bb10  _CLA1_INT7_ISR                        
0     0000bb1a  _CLA1_INT8_ISR                        
1     00001400  _Cla1Regs                             
1     00006400  _Comp1Regs                            
1     00006420  _Comp2Regs                            
1     00006440  _Comp3Regs                            
0     00008000  _ConfigDescAlloc                      
0     00008051  _ConfigDescFree                       
0     0000bf5c  _ControlHandler                       
1     00000c00  _CpuTimer0Regs                        
1     00000c08  _CpuTimer1Regs                        
1     00000c10  _CpuTimer2Regs                        
1     003f7ff8  _CsmPwl                               
1     00000ae0  _CsmRegs                              
0     0000b7dc  _DATALOG_ISR                          
0     0000ba0c  _DINTCH1_ISR                          
0     0000ba16  _DINTCH2_ISR                          
0     0000ba20  _DINTCH3_ISR                          
0     0000ba2a  _DINTCH4_ISR                          
0     0000ba34  _DINTCH5_ISR                          
0     0000ba3e  _DINTCH6_ISR                          
0     0000d59f  _DSP28x_usDelay                       
1     00000880  _DevEmuRegs                           
1     00001000  _DmaRegs                              
0     0000ba84  _ECAN0INTA_ISR                        
0     0000ba8e  _ECAN1INTA_ISR                        
0     0000b96c  _ECAP1_INT_ISR                        
0     0000b976  _ECAP2_INT_ISR                        
0     0000b980  _ECAP3_INT_ISR                        
1     00006040  _ECanaLAMRegs                         
1     000060c0  _ECanaMOTORegs                        
1     00006080  _ECanaMOTSRegs                        
1     00006100  _ECanaMboxes                          
1     00006000  _ECanaRegs                            
1     00006a00  _ECap1Regs                            
1     00006a20  _ECap2Regs                            
1     00006a40  _ECap3Regs                            
0     0000bb42  _EMPTY_ISR                            
0     0000b7f0  _EMUINT_ISR                           
0     0000b91c  _EPWM1_INT_ISR                        
0     0000b8cc  _EPWM1_TZINT_ISR                      
0     0000b926  _EPWM2_INT_ISR                        
0     0000b8d6  _EPWM2_TZINT_ISR                      
0     0000b930  _EPWM3_INT_ISR                        
0     0000b8e0  _EPWM3_TZINT_ISR                      
0     0000b93a  _EPWM4_INT_ISR                        
0     0000b8ea  _EPWM4_TZINT_ISR                      
0     0000b944  _EPWM5_INT_ISR                        
0     0000b8f4  _EPWM5_TZINT_ISR                      
0     0000b94e  _EPWM6_INT_ISR                        
0     0000b8fe  _EPWM6_TZINT_ISR                      
0     0000b958  _EPWM7_INT_ISR                        
0     0000b908  _EPWM7_TZINT_ISR                      
0     0000b962  _EPWM8_INT_ISR                        
0     0000b912  _EPWM8_TZINT_ISR                      
1     00006800  _EPwm1Regs                            
1     00006840  _EPwm2Regs                            
1     00006880  _EPwm3Regs                            
1     000068c0  _EPwm4Regs                            
1     00006900  _EPwm5Regs                            
1     00006940  _EPwm6Regs                            
1     00006980  _EPwm7Regs                            
1     000069c0  _EPwm8Regs                            
0     0000b99e  _EQEP1_INT_ISR                        
0     0000b9a8  _EQEP2_INT_ISR                        
1     00006b00  _EQep1Regs                            
1     00006b40  _EQep2Regs                            
1     00000d01  _EmuBMode                             
1     00000d00  _EmuKey                               
0     0000d49b  _EnableInterrupts                     
1     00000a80  _FlashRegs                            
1     00000d04  _Flash_CPUScaleFactor                 
1     00000d02  _Flash_CallbackPtr                    
1     00006f80  _GpioCtrlRegs                         
1     00006fc0  _GpioDataRegs                         
1     00006fe0  _GpioIntRegs                          
0     0000b98a  _HRCAP1_INT_ISR                       
0     0000b994  _HRCAP2_INT_ISR                       
0     0000b9b2  _HRCAP3_INT_ISR                       
0     0000b9bc  _HRCAP4_INT_ISR                       
1     00006ac0  _HRCap1Regs                           
1     00006ae0  _HRCap2Regs                           
1     00006c80  _HRCap3Regs                           
1     00006ca0  _HRCap4Regs                           
0     0000ba48  _I2CINT1A_ISR                         
0     0000ba52  _I2CINT2A_ISR                         
1     00007900  _I2caRegs                             
0     0000b804  _ILLEGAL_ISR                          
0     0000b7c8  _INT13_ISR                            
0     0000b7d2  _INT14_ISR                            
0     0000d47c  _InitPieCtrl                          
0     0000d4a4  _InitPieVectTable                     
0     0000d589  _IntDefaultHandler                    
0     0000ca47  _IntDisable                           
0     0000ca20  _IntEnable                            
0     0000c9de  _IntMasterDisable                     
0     0000c9da  _IntMasterEnable                      
0     0000c9e2  _IntRegister                          
0     0000ca00  _IntUnregister                        
0     000090e9  _InternalUSBHCDSendEvent              
0     0000d352  _InternalUSBRegisterTickHandler       
0     0000d380  _InternalUSBStartOfFrameTick          
0     0000d329  _InternalUSBTickInit                  
0     0000d34e  _InternalUSBTickReset                 
0     0000cb2c  _Interrupt_disable                    
0     0000cae2  _Interrupt_enable                     
0     0000bb38  _LUF_ISR                              
0     0000bb2e  _LVF_ISR                              
0     0000b9f8  _MRINTA_ISR                           
0     0000ba02  _MXINTA_ISR                           
1     00005000  _McbspaRegs                           
0     0000b7fa  _NMI_ISR                              
1     00007060  _NmiIntruptRegs                       
0     0000c781  _OTGDeviceDisconnect                  
0     0000bb4f  _PIE_RESERVED                         
1     003d7e80  _PartIdRegs                           
1     00000ce0  _PieCtrlRegs                          
1     00000d00  _PieVectTable                         
1     0000e7c0  _PieVectTableInit                     
0     0000adc4  _ProcessDataFromHost                  
0     0000ae51  _ProcessDataToHost                    
0     0000ae22  _ProcessNotificationToHost            
0     0000b7e6  _RTOSINT_ISR                          
0     0000bfad  _RxHandler                            
0     0000ba5c  _SCIRXINTA_ISR                        
0     0000ba70  _SCIRXINTB_ISR                        
0     0000ba66  _SCITXINTA_ISR                        
0     0000ba7a  _SCITXINTB_ISR                        
0     0000b9d0  _SPIRXINTA_ISR                        
0     0000b9e4  _SPIRXINTB_ISR                        
0     0000b9da  _SPITXINTA_ISR                        
0     0000b9ee  _SPITXINTB_ISR                        
1     00007050  _SciaRegs                             
1     00007750  _ScibRegs                             
1     00007040  _SpiaRegs                             
1     00007740  _SpibRegs                             
0     0000d03c  _SysCtlClockGet                       
0     0000d02b  _SysCtlDelay                          
0     0000cfea  _SysCtlPeripheralDisable              
0     0000cfae  _SysCtlPeripheralEnable               
0     0000d026  _SysCtlPeripheralPresent              
0     0000cfaa  _SysCtlPeripheralReset                
0     0000d051  _SysCtlUSBPLLDisable                  
0     0000d044  _SysCtlUSBPLLEnable                   
0     0000bfd9  _SysCtrlInit                          
1     00007010  _SysCtrlRegs                          
1     00000985  _SysPwrCtrlRegs                       
0     0000b8b8  _TINT0_ISR                            
0     0000bfa5  _TxHandler                            
0     0000c1f0  _UARTBusy                             
0     0000c1b7  _UARTCharGet                          
0     0000c1a6  _UARTCharGetNonBlocking               
0     0000c1e0  _UARTCharPut                          
0     0000c1cd  _UARTCharPutNonBlocking               
0     0000c18c  _UARTCharsAvail                       
0     0000c11c  _UARTConfigGetExpClk                  
0     0000c0e5  _UARTConfigSetExpClk                  
0     0000c14a  _UARTDisable                          
0     0000c140  _UARTEnable                           
0     0000c169  _UARTFIFODisable                      
0     0000c160  _UARTFIFOEnable                       
0     0000c0cf  _UARTFIFOLevelGet                     
0     0000c0b5  _UARTFIFOLevelSet                     
0     0000c2e8  _UARTIntClear                         
0     0000c282  _UARTIntDisable                       
0     0000c251  _UARTIntEnable                        
0     0000c2b8  _UARTIntStatus                        
0     0000c0ac  _UARTParityModeGet                    
0     0000c0a2  _UARTParityModeSet                    
0     0000c1fd  _UARTRXIntRegister                    
0     0000c229  _UARTRXIntUnregister                  
0     0000c31b  _UARTRxErrorClear                     
0     0000c315  _UARTRxErrorGet                       
0     0000c199  _UARTSpaceAvail                       
0     0000bb63  _UARTStdioInit                        
0     0000bb6d  _UARTStdioInitExpClk                  
0     0000c213  _UARTTXIntRegister                    
0     0000c23d  _UARTTXIntUnregister                  
0     0000c182  _UARTTxIntModeGet                     
0     0000c172  _UARTTxIntModeSet                     
0     0000bc56  _UARTgetc                             
0     0000bbea  _UARTgets                             
0     0000bc5c  _UARTprintf                           
0     0000bbb5  _UARTwrite                            
0     0000d569  _USB0DeviceIntHandler                 
0     0000c5d8  _USB0DualModeIntHandler               
0     0000906f  _USB0HostIntHandler                   
0     0000c702  _USB0OTGModeIntHandler                
0     0000b9c6  _USB0_INT_ISR                         
0     0000c4ec  _USBBufferCallbackDataSet             
0     0000c53c  _USBBufferDataAvailable               
0     0000c4dc  _USBBufferDataRemoved                 
0     0000c4c9  _USBBufferDataWritten                 
0     0000c554  _USBBufferEventCallback               
0     0000c514  _USBBufferFlush                       
0     0000c4bb  _USBBufferInfoGet                     
0     0000c48a  _USBBufferInit                        
0     0000c520  _USBBufferRead                        
0     0000c548  _USBBufferSpaceAvailable              
0     0000c4f6  _USBBufferWrite                       
0     0000c4a4  _USBBufferZeroLengthPacketInsert      
0     0000b17c  _USBDCDCCompositeInit                 
0     0000b214  _USBDCDCInit                          
0     0000b2e9  _USBDCDCPacketRead                    
0     0000b2a4  _USBDCDCPacketWrite                   
0     0000b3ba  _USBDCDCPowerStatusSet                
0     0000b3c3  _USBDCDCRemoteWakeupRequest           
0     0000b361  _USBDCDCRxPacketAvailable             
0     0000b38c  _USBDCDCSerialStateChange             
0     0000b274  _USBDCDCSetControlCBData              
0     0000b280  _USBDCDCSetRxCBData                   
0     0000b292  _USBDCDCSetTxCBData                   
0     0000b267  _USBDCDCTerm                          
0     0000b351  _USBDCDCTxPacketAvailable             
0     0000cc14  _USBDCDConfigDescGet                  
0     0000cbef  _USBDCDConfigDescGetNum               
0     0000cbd6  _USBDCDConfigDescGetSize              
0     0000cc7d  _USBDCDConfigGetInterface             
0     0000cc96  _USBDCDConfigGetInterfaceEndpoint     
0     0000cc58  _USBDCDConfigGetNumAlternateInterfaces
0     0000a464  _USBDCDDeviceInfoInit                 
0     0000a474  _USBDCDInit                           
0     0000a55b  _USBDCDPowerStatusSet                 
0     0000a568  _USBDCDRemoteWakeupRequest            
0     0000a525  _USBDCDRequestDataEP0                 
0     0000a533  _USBDCDSendDataEP0                    
0     0000a542  _USBDCDSetDefaultConfiguration        
0     0000a54a  _USBDCDStallEP0                       
0     0000a4f2  _USBDCDTerm                           
0     0000d411  _USBDelay                             
0     0000cf05  _USBDescGet                           
0     0000cf7e  _USBDescGetInterface                  
0     0000cf98  _USBDescGetInterfaceEndpoint          
0     0000cedf  _USBDescGetNum                        
0     0000cf30  _USBDescGetNumAlternateInterfaces     
0     00009bc0  _USBDevAddrGet                        
0     00009bad  _USBDevAddrSet                        
0     00009b80  _USBDevConnect                        
0     00009b96  _USBDevDisconnect                     
0     00009d2d  _USBDevEndpointConfigGet              
0     00009ca4  _USBDevEndpointConfigSet              
0     00009f74  _USBDevEndpointDataAck                
0     00009ab7  _USBDevEndpointStall                  
0     00009b12  _USBDevEndpointStallClear             
0     00009992  _USBDevEndpointStatusClear            
0     0000a40d  _USBDevMode                           
0     0000c834  _USBDeviceConfig                      
0     0000c971  _USBDeviceConfigAlternate             
0     0000a5eb  _USBDeviceEnumHandler                 
0     0000a6a9  _USBDeviceEnumResetHandler            
0     0000ac0a  _USBDeviceIntHandlerInternal          
0     0000a57e  _USBDeviceResumeTickHandler           
0     0000c612  _USBDualModeInit                      
0     0000c655  _USBDualModeTerm                      
0     0000a3b0  _USBEndpointDMAChannel                
0     00009eaa  _USBEndpointDMADisable                
0     00009e92  _USBEndpointDMAEnable                 
0     00009ec4  _USBEndpointDataAvail                 
0     00009f0a  _USBEndpointDataGet                   
0     0000a001  _USBEndpointDataPut                   
0     0000a055  _USBEndpointDataSend                  
0     00009a77  _USBEndpointDataToggleClear           
0     0000a450  _USBEndpointPacketCountSet            
0     00009903  _USBEndpointStatus                    
0     0000a390  _USBFIFOAddrGet                       
0     00009e2a  _USBFIFOConfigGet                     
0     00009dc4  _USBFIFOConfigSet                     
0     0000a0ae  _USBFIFOFlush                         
0     0000a35b  _USBFrameNumberGet                    
0     0000d409  _USBGPIODisable                       
0     0000d401  _USBGPIOEnable                        
0     00009355  _USBHCDControlTransfer                
0     0000954c  _USBHCDDevAddress                     
0     00009560  _USBHCDDevClass                       
0     00009538  _USBHCDDevHubPort                     
0     000095aa  _USBHCDDevProtocol                    
0     00009585  _USBHCDDevSubClass                    
0     000080d3  _USBHCDEventDisable                   
0     000080be  _USBHCDEventEnable                    
0     000093e7  _USBHCDHubDeviceConnected             
0     0000943d  _USBHCDHubDeviceDisconnected          
0     000089cc  _USBHCDInit                           
0     00009195  _USBHCDMain                           
0     00008397  _USBHCDPipeAlloc                      
0     000081a1  _USBHCDPipeAllocSize                  
0     000083a6  _USBHCDPipeConfig                     
0     0000864d  _USBHCDPipeDataAck                    
0     0000877f  _USBHCDPipeFree                       
0     0000866a  _USBHCDPipeRead                       
0     00008622  _USBHCDPipeReadNonBlocking            
0     0000857b  _USBHCDPipeSchedule                   
0     00008476  _USBHCDPipeStatus                     
0     0000847b  _USBHCDPipeWrite                      
0     000089c1  _USBHCDPowerAutomatic                 
0     00008990  _USBHCDPowerConfigGet                 
0     00008988  _USBHCDPowerConfigInit                
0     00008997  _USBHCDPowerConfigSet                 
0     00008a1d  _USBHCDRegisterDrivers                
0     00008a88  _USBHCDReset                          
0     00008ab7  _USBHCDResume                         
0     00008b75  _USBHCDSetAddress                     
0     00008c1e  _USBHCDSetConfig                      
0     00008c42  _USBHCDSetInterface                   
0     00008aae  _USBHCDSuspend                        
0     00008a28  _USBHCDTerm                           
0     0000b7b4  _USBHHubClose                         
0     0000b784  _USBHHubEnumerationComplete           
0     0000b795  _USBHHubEnumerationError              
0     0000b7bd  _USBHHubInit                          
0     0000b697  _USBHHubMain                          
0     0000b7a6  _USBHHubOpen                          
0     0000a1e9  _USBHostAddrGet                       
0     0000a1a7  _USBHostAddrSet                       
0     00008c6e  _USBHostCheckPipes                    
0     00009bd4  _USBHostEndpointConfig                
0     00009fbe  _USBHostEndpointDataAck               
0     000099fc  _USBHostEndpointDataToggle            
0     00009942  _USBHostEndpointStatusClear           
0     0000a285  _USBHostHubAddrGet                    
0     0000a22d  _USBHostHubAddrSet                    
0     00008cf9  _USBHostIntHandlerInternal            
0     0000a3f6  _USBHostMode                          
0     0000a2c9  _USBHostPwrConfig                     
0     0000a344  _USBHostPwrDisable                    
0     0000a32d  _USBHostPwrEnable                     
0     0000a316  _USBHostPwrFaultDisable               
0     0000a2ff  _USBHostPwrFaultEnable                
0     0000a112  _USBHostRequestIN                     
0     0000a150  _USBHostRequestINClear                
0     0000a190  _USBHostRequestStatus                 
0     00009672  _USBHostReset                         
0     00009691  _USBHostResume                        
0     000096b2  _USBHostSpeedGet                      
0     0000965e  _USBHostSuspend                       
0     00009724  _USBIntDisable                        
0     000097df  _USBIntDisableControl                 
0     00009883  _USBIntDisableEndpoint                
0     00009783  _USBIntEnable                         
0     0000981a  _USBIntEnableControl                  
0     000098a1  _USBIntEnableEndpoint                 
0     000098d5  _USBIntRegister                       
0     000096d5  _USBIntStatus                         
0     00009852  _USBIntStatusControl                  
0     000098bd  _USBIntStatusEndpoint                 
0     000098ed  _USBIntUnregister                     
0     0000ce86  _USBLibDMAInit                        
0     0000a399  _USBModeGet                           
0     0000a45f  _USBNumEndpointsGet                   
0     0000c78f  _USBOTGMain                           
0     0000a424  _USBOTGMode                           
0     0000c68a  _USBOTGModeInit                       
0     0000c66e  _USBOTGModeTerm                       
0     0000c6fa  _USBOTGPollRate                       
0     0000a36f  _USBOTGSessionRequest                 
0     0000a43b  _USBPHYPowerOff                       
0     0000a445  _USBPHYPowerOn                        
0     0000cd98  _USBRingBufAdvanceRead                
0     0000cdae  _USBRingBufAdvanceWrite               
0     0000cd4d  _USBRingBufContigFree                 
0     0000cd3e  _USBRingBufContigUsed                 
0     0000ccfe  _USBRingBufEmpty                      
0     0000cd10  _USBRingBufFlush                      
0     0000cd33  _USBRingBufFree                       
0     0000cce5  _USBRingBufFull                       
0     0000cdfe  _USBRingBufInit                       
0     0000cd7f  _USBRingBufRead                       
0     0000cd6c  _USBRingBufReadOne                    
0     0000cd67  _USBRingBufSize                       
0     0000cd23  _USBRingBufUsed                       
0     0000cde6  _USBRingBufWrite                      
0     0000cdd2  _USBRingBufWriteOne                   
0     0000c5c2  _USBStackModeSet                      
0     0000d13b  _USBUARTRXIntHandler                  
0     0000d0f2  _USBUARTTXIntHandler                  
0     0000b868  _USER10_ISR                           
0     0000b872  _USER11_ISR                           
0     0000b87c  _USER12_ISR                           
0     0000b80e  _USER1_ISR                            
0     0000b818  _USER2_ISR                            
0     0000b822  _USER3_ISR                            
0     0000b82c  _USER4_ISR                            
0     0000b836  _USER5_ISR                            
0     0000b840  _USER6_ISR                            
0     0000b84a  _USER7_ISR                            
0     0000b854  _USER8_ISR                            
0     0000b85e  _USER9_ISR                            
1     00004000  _Usb0Regs                             
0     0000b8c2  _WAKEINT_ISR                          
0     0000b89a  _XINT1_ISR                            
0     0000b8a4  _XINT2_ISR                            
0     0000bb24  _XINT3_ISR                            
1     00007070  _XIntruptRegs                         
1     00000800  __STACK_END                           
abs   00000400  __STACK_SIZE                          
1     0000e6f6  ___TI_cleanup_ptr                     
1     0000e6f8  ___TI_dtors_ptr                       
1     0000e6f4  ___TI_enable_exit_profile_output      
abs   ffffffff  ___TI_pprof_out_hndl                  
abs   ffffffff  ___TI_prof_data_size                  
abs   ffffffff  ___TI_prof_data_start                 
abs   ffffffff  ___binit__                            
abs   ffffffff  ___c_args__                           
0     00000050  ___cinit__                            
0     0000be11  ___error__                            
0     0000d5a6  ___etext__                            
abs   ffffffff  ___pinit__                            
0     00008000  ___text__                             
0     0000d527  __args_main                           
1     0000e6fe  __lock                                
0     0000d59e  __nop                                 
0     0000d59a  __register_lock                       
0     0000d596  __register_unlock                     
1     00000400  __stack                               
0     0000d5a5  __system_post_cinit                   
0     0000d5a3  __system_pre_init                     
1     0000e7be  __unlock                              
0     0000d453  _abort                                
0     0000d3ab  _c_int00                              
0     0000d4ca  _copy_in                              
abs   000007c0  _ebss_size                            
1     0000e000  _ebss_start                           
0     0000d455  _exit                                 
0     0000d188  _f28x_USB0DeviceIntHandler            
0     0000d1ea  _f28x_USB0DualModeIntHandler          
0     0000d1b9  _f28x_USB0HostIntHandler              
1     0000e6cc  _g_bUSBTimerInitialized               
1     0000e6ec  _g_eOTGModeState                      
1     0000e6eb  _g_iUSBMode                           
1     0000ead2  _g_pCDCCompSerConfigDescriptors       
1     0000e6d2  _g_pfnTickHandlers                    
1     0000e440  _g_pi8USBRxBuffer                     
1     0000e540  _g_pi8USBTxBuffer                     
1     0000ead4  _g_ppCDCSerConfigDescriptors          
1     0000e700  _g_ppsDevInfo                         
1     0000e394  _g_psCDCCompSerSections               
1     0000e38e  _g_psCDCSerSections                   
1     0000e704  _g_psDCDInst                          
1     0000e9c6  _g_pui8CDCSerCommInterface            
1     0000ea3e  _g_pui8CDCSerDataInterface            
1     0000e3a4  _g_pui8CDCSerDescriptor               
1     0000e3ad  _g_pui8CDCSerDeviceDescriptor         
1     0000e90d  _g_pui8ConfigString                   
1     0000e976  _g_pui8ControlInterfaceString         
1     0000e39c  _g_pui8IADSerDescriptor               
1     0000eab4  _g_pui8LangDescriptor                 
1     0000e9a2  _g_pui8ManufacturerString             
1     0000e9e9  _g_pui8ProdectString                  
1     0000e3d8  _g_pui8RxBufferWorkspace              
1     0000ea55  _g_pui8SerialNumberString             
1     0000ea9c  _g_pui8StringDescriptors              
1     0000e3c0  _g_pui8TxBufferWorkspace              
1     0000e6de  _g_pvTickInstance                     
1     0000eab8  _g_sCDCCompSerConfigHeader            
1     0000e400  _g_sCDCDevice                         
1     0000ea26  _g_sCDCHandlers                       
1     0000eabc  _g_sCDCSerCommInterfaceSection        
1     0000eac0  _g_sCDCSerConfigHeader                
1     0000eac4  _g_sCDCSerConfigSection               
1     0000eac8  _g_sCDCSerDataInterfaceSection        
1     0000eacc  _g_sIADSerConfigSection               
1     0000ea68  _g_sRxBuffer                          
1     0000ea7a  _g_sTxBuffer                          
1     0000e6ce  _g_ui32CurrentUSBTick                 
1     0000e6f0  _g_ui32PollRate                       
1     0000e6d0  _g_ui32USBSOFCount                    
1     0000e6f2  _g_ui32WaitTicks                      
0     0000c00b  _main                                 
0     0000d4ee  _memcpy                               
0     0000bb59  _rsvd_ISR                             
abs   ffffffff  binit                                 
0     00000050  cinit                                 
0     00000000  code_start                            
0     0000d5a6  etext                                 
abs   ffffffff  pinit                                 


GLOBAL SYMBOLS: SORTED BY Symbol Address 

page  address   name                                  
----  -------   ----                                  
0     00000000  code_start                            
0     00000050  ___cinit__                            
0     00000050  cinit                                 
0     00008000  .text                                 
0     00008000  _ConfigDescAlloc                      
0     00008000  ___text__                             
0     00008051  _ConfigDescFree                       
0     000080be  _USBHCDEventEnable                    
0     000080d3  _USBHCDEventDisable                   
0     000081a1  _USBHCDPipeAllocSize                  
0     00008397  _USBHCDPipeAlloc                      
0     000083a6  _USBHCDPipeConfig                     
0     00008476  _USBHCDPipeStatus                     
0     0000847b  _USBHCDPipeWrite                      
0     0000857b  _USBHCDPipeSchedule                   
0     00008622  _USBHCDPipeReadNonBlocking            
0     0000864d  _USBHCDPipeDataAck                    
0     0000866a  _USBHCDPipeRead                       
0     0000877f  _USBHCDPipeFree                       
0     00008988  _USBHCDPowerConfigInit                
0     00008990  _USBHCDPowerConfigGet                 
0     00008997  _USBHCDPowerConfigSet                 
0     000089c1  _USBHCDPowerAutomatic                 
0     000089cc  _USBHCDInit                           
0     00008a1d  _USBHCDRegisterDrivers                
0     00008a28  _USBHCDTerm                           
0     00008a88  _USBHCDReset                          
0     00008aae  _USBHCDSuspend                        
0     00008ab7  _USBHCDResume                         
0     00008b75  _USBHCDSetAddress                     
0     00008c1e  _USBHCDSetConfig                      
0     00008c42  _USBHCDSetInterface                   
0     00008c6e  _USBHostCheckPipes                    
0     00008cf9  _USBHostIntHandlerInternal            
0     0000906f  _USB0HostIntHandler                   
0     000090e9  _InternalUSBHCDSendEvent              
0     00009195  _USBHCDMain                           
0     00009355  _USBHCDControlTransfer                
0     000093e7  _USBHCDHubDeviceConnected             
0     0000943d  _USBHCDHubDeviceDisconnected          
0     00009538  _USBHCDDevHubPort                     
0     0000954c  _USBHCDDevAddress                     
0     00009560  _USBHCDDevClass                       
0     00009585  _USBHCDDevSubClass                    
0     000095aa  _USBHCDDevProtocol                    
0     0000965e  _USBHostSuspend                       
0     00009672  _USBHostReset                         
0     00009691  _USBHostResume                        
0     000096b2  _USBHostSpeedGet                      
0     000096d5  _USBIntStatus                         
0     00009724  _USBIntDisable                        
0     00009783  _USBIntEnable                         
0     000097df  _USBIntDisableControl                 
0     0000981a  _USBIntEnableControl                  
0     00009852  _USBIntStatusControl                  
0     00009883  _USBIntDisableEndpoint                
0     000098a1  _USBIntEnableEndpoint                 
0     000098bd  _USBIntStatusEndpoint                 
0     000098d5  _USBIntRegister                       
0     000098ed  _USBIntUnregister                     
0     00009903  _USBEndpointStatus                    
0     00009942  _USBHostEndpointStatusClear           
0     00009992  _USBDevEndpointStatusClear            
0     000099fc  _USBHostEndpointDataToggle            
0     00009a77  _USBEndpointDataToggleClear           
0     00009ab7  _USBDevEndpointStall                  
0     00009b12  _USBDevEndpointStallClear             
0     00009b80  _USBDevConnect                        
0     00009b96  _USBDevDisconnect                     
0     00009bad  _USBDevAddrSet                        
0     00009bc0  _USBDevAddrGet                        
0     00009bd4  _USBHostEndpointConfig                
0     00009ca4  _USBDevEndpointConfigSet              
0     00009d2d  _USBDevEndpointConfigGet              
0     00009dc4  _USBFIFOConfigSet                     
0     00009e2a  _USBFIFOConfigGet                     
0     00009e92  _USBEndpointDMAEnable                 
0     00009eaa  _USBEndpointDMADisable                
0     00009ec4  _USBEndpointDataAvail                 
0     00009f0a  _USBEndpointDataGet                   
0     00009f74  _USBDevEndpointDataAck                
0     00009fbe  _USBHostEndpointDataAck               
0     0000a001  _USBEndpointDataPut                   
0     0000a055  _USBEndpointDataSend                  
0     0000a0ae  _USBFIFOFlush                         
0     0000a112  _USBHostRequestIN                     
0     0000a150  _USBHostRequestINClear                
0     0000a190  _USBHostRequestStatus                 
0     0000a1a7  _USBHostAddrSet                       
0     0000a1e9  _USBHostAddrGet                       
0     0000a22d  _USBHostHubAddrSet                    
0     0000a285  _USBHostHubAddrGet                    
0     0000a2c9  _USBHostPwrConfig                     
0     0000a2ff  _USBHostPwrFaultEnable                
0     0000a316  _USBHostPwrFaultDisable               
0     0000a32d  _USBHostPwrEnable                     
0     0000a344  _USBHostPwrDisable                    
0     0000a35b  _USBFrameNumberGet                    
0     0000a36f  _USBOTGSessionRequest                 
0     0000a390  _USBFIFOAddrGet                       
0     0000a399  _USBModeGet                           
0     0000a3b0  _USBEndpointDMAChannel                
0     0000a3f6  _USBHostMode                          
0     0000a40d  _USBDevMode                           
0     0000a424  _USBOTGMode                           
0     0000a43b  _USBPHYPowerOff                       
0     0000a445  _USBPHYPowerOn                        
0     0000a450  _USBEndpointPacketCountSet            
0     0000a45f  _USBNumEndpointsGet                   
0     0000a464  _USBDCDDeviceInfoInit                 
0     0000a474  _USBDCDInit                           
0     0000a4f2  _USBDCDTerm                           
0     0000a525  _USBDCDRequestDataEP0                 
0     0000a533  _USBDCDSendDataEP0                    
0     0000a542  _USBDCDSetDefaultConfiguration        
0     0000a54a  _USBDCDStallEP0                       
0     0000a55b  _USBDCDPowerStatusSet                 
0     0000a568  _USBDCDRemoteWakeupRequest            
0     0000a57e  _USBDeviceResumeTickHandler           
0     0000a5eb  _USBDeviceEnumHandler                 
0     0000a6a9  _USBDeviceEnumResetHandler            
0     0000ac0a  _USBDeviceIntHandlerInternal          
0     0000adc4  _ProcessDataFromHost                  
0     0000ae22  _ProcessNotificationToHost            
0     0000ae51  _ProcessDataToHost                    
0     0000b17c  _USBDCDCCompositeInit                 
0     0000b214  _USBDCDCInit                          
0     0000b267  _USBDCDCTerm                          
0     0000b274  _USBDCDCSetControlCBData              
0     0000b280  _USBDCDCSetRxCBData                   
0     0000b292  _USBDCDCSetTxCBData                   
0     0000b2a4  _USBDCDCPacketWrite                   
0     0000b2e9  _USBDCDCPacketRead                    
0     0000b351  _USBDCDCTxPacketAvailable             
0     0000b361  _USBDCDCRxPacketAvailable             
0     0000b38c  _USBDCDCSerialStateChange             
0     0000b3ba  _USBDCDCPowerStatusSet                
0     0000b3c3  _USBDCDCRemoteWakeupRequest           
0     0000b697  _USBHHubMain                          
0     0000b784  _USBHHubEnumerationComplete           
0     0000b795  _USBHHubEnumerationError              
0     0000b7a6  _USBHHubOpen                          
0     0000b7b4  _USBHHubClose                         
0     0000b7bd  _USBHHubInit                          
0     0000b7c8  _INT13_ISR                            
0     0000b7d2  _INT14_ISR                            
0     0000b7dc  _DATALOG_ISR                          
0     0000b7e6  _RTOSINT_ISR                          
0     0000b7f0  _EMUINT_ISR                           
0     0000b7fa  _NMI_ISR                              
0     0000b804  _ILLEGAL_ISR                          
0     0000b80e  _USER1_ISR                            
0     0000b818  _USER2_ISR                            
0     0000b822  _USER3_ISR                            
0     0000b82c  _USER4_ISR                            
0     0000b836  _USER5_ISR                            
0     0000b840  _USER6_ISR                            
0     0000b84a  _USER7_ISR                            
0     0000b854  _USER8_ISR                            
0     0000b85e  _USER9_ISR                            
0     0000b868  _USER10_ISR                           
0     0000b872  _USER11_ISR                           
0     0000b87c  _USER12_ISR                           
0     0000b886  _ADCINT1_ISR                          
0     0000b890  _ADCINT2_ISR                          
0     0000b89a  _XINT1_ISR                            
0     0000b8a4  _XINT2_ISR                            
0     0000b8ae  _ADCINT9_ISR                          
0     0000b8b8  _TINT0_ISR                            
0     0000b8c2  _WAKEINT_ISR                          
0     0000b8cc  _EPWM1_TZINT_ISR                      
0     0000b8d6  _EPWM2_TZINT_ISR                      
0     0000b8e0  _EPWM3_TZINT_ISR                      
0     0000b8ea  _EPWM4_TZINT_ISR                      
0     0000b8f4  _EPWM5_TZINT_ISR                      
0     0000b8fe  _EPWM6_TZINT_ISR                      
0     0000b908  _EPWM7_TZINT_ISR                      
0     0000b912  _EPWM8_TZINT_ISR                      
0     0000b91c  _EPWM1_INT_ISR                        
0     0000b926  _EPWM2_INT_ISR                        
0     0000b930  _EPWM3_INT_ISR                        
0     0000b93a  _EPWM4_INT_ISR                        
0     0000b944  _EPWM5_INT_ISR                        
0     0000b94e  _EPWM6_INT_ISR                        
0     0000b958  _EPWM7_INT_ISR                        
0     0000b962  _EPWM8_INT_ISR                        
0     0000b96c  _ECAP1_INT_ISR                        
0     0000b976  _ECAP2_INT_ISR                        
0     0000b980  _ECAP3_INT_ISR                        
0     0000b98a  _HRCAP1_INT_ISR                       
0     0000b994  _HRCAP2_INT_ISR                       
0     0000b99e  _EQEP1_INT_ISR                        
0     0000b9a8  _EQEP2_INT_ISR                        
0     0000b9b2  _HRCAP3_INT_ISR                       
0     0000b9bc  _HRCAP4_INT_ISR                       
0     0000b9c6  _USB0_INT_ISR                         
0     0000b9d0  _SPIRXINTA_ISR                        
0     0000b9da  _SPITXINTA_ISR                        
0     0000b9e4  _SPIRXINTB_ISR                        
0     0000b9ee  _SPITXINTB_ISR                        
0     0000b9f8  _MRINTA_ISR                           
0     0000ba02  _MXINTA_ISR                           
0     0000ba0c  _DINTCH1_ISR                          
0     0000ba16  _DINTCH2_ISR                          
0     0000ba20  _DINTCH3_ISR                          
0     0000ba2a  _DINTCH4_ISR                          
0     0000ba34  _DINTCH5_ISR                          
0     0000ba3e  _DINTCH6_ISR                          
0     0000ba48  _I2CINT1A_ISR                         
0     0000ba52  _I2CINT2A_ISR                         
0     0000ba5c  _SCIRXINTA_ISR                        
0     0000ba66  _SCITXINTA_ISR                        
0     0000ba70  _SCIRXINTB_ISR                        
0     0000ba7a  _SCITXINTB_ISR                        
0     0000ba84  _ECAN0INTA_ISR                        
0     0000ba8e  _ECAN1INTA_ISR                        
0     0000ba98  _ADCINT3_ISR                          
0     0000baa2  _ADCINT4_ISR                          
0     0000baac  _ADCINT5_ISR                          
0     0000bab6  _ADCINT6_ISR                          
0     0000bac0  _ADCINT7_ISR                          
0     0000baca  _ADCINT8_ISR                          
0     0000bad4  _CLA1_INT1_ISR                        
0     0000bade  _CLA1_INT2_ISR                        
0     0000bae8  _CLA1_INT3_ISR                        
0     0000baf2  _CLA1_INT4_ISR                        
0     0000bafc  _CLA1_INT5_ISR                        
0     0000bb06  _CLA1_INT6_ISR                        
0     0000bb10  _CLA1_INT7_ISR                        
0     0000bb1a  _CLA1_INT8_ISR                        
0     0000bb24  _XINT3_ISR                            
0     0000bb2e  _LVF_ISR                              
0     0000bb38  _LUF_ISR                              
0     0000bb42  _EMPTY_ISR                            
0     0000bb4f  _PIE_RESERVED                         
0     0000bb59  _rsvd_ISR                             
0     0000bb63  _UARTStdioInit                        
0     0000bb6d  _UARTStdioInitExpClk                  
0     0000bbb5  _UARTwrite                            
0     0000bbea  _UARTgets                             
0     0000bc56  _UARTgetc                             
0     0000bc5c  _UARTprintf                           
0     0000be11  ___error__                            
0     0000bf5c  _ControlHandler                       
0     0000bfa5  _TxHandler                            
0     0000bfad  _RxHandler                            
0     0000bfd9  _SysCtrlInit                          
0     0000c00b  _main                                 
0     0000c0a2  _UARTParityModeSet                    
0     0000c0ac  _UARTParityModeGet                    
0     0000c0b5  _UARTFIFOLevelSet                     
0     0000c0cf  _UARTFIFOLevelGet                     
0     0000c0e5  _UARTConfigSetExpClk                  
0     0000c11c  _UARTConfigGetExpClk                  
0     0000c140  _UARTEnable                           
0     0000c14a  _UARTDisable                          
0     0000c160  _UARTFIFOEnable                       
0     0000c169  _UARTFIFODisable                      
0     0000c172  _UARTTxIntModeSet                     
0     0000c182  _UARTTxIntModeGet                     
0     0000c18c  _UARTCharsAvail                       
0     0000c199  _UARTSpaceAvail                       
0     0000c1a6  _UARTCharGetNonBlocking               
0     0000c1b7  _UARTCharGet                          
0     0000c1cd  _UARTCharPutNonBlocking               
0     0000c1e0  _UARTCharPut                          
0     0000c1f0  _UARTBusy                             
0     0000c1fd  _UARTRXIntRegister                    
0     0000c213  _UARTTXIntRegister                    
0     0000c229  _UARTRXIntUnregister                  
0     0000c23d  _UARTTXIntUnregister                  
0     0000c251  _UARTIntEnable                        
0     0000c282  _UARTIntDisable                       
0     0000c2b8  _UARTIntStatus                        
0     0000c2e8  _UARTIntClear                         
0     0000c315  _UARTRxErrorGet                       
0     0000c31b  _UARTRxErrorClear                     
0     0000c48a  _USBBufferInit                        
0     0000c4a4  _USBBufferZeroLengthPacketInsert      
0     0000c4bb  _USBBufferInfoGet                     
0     0000c4c9  _USBBufferDataWritten                 
0     0000c4dc  _USBBufferDataRemoved                 
0     0000c4ec  _USBBufferCallbackDataSet             
0     0000c4f6  _USBBufferWrite                       
0     0000c514  _USBBufferFlush                       
0     0000c520  _USBBufferRead                        
0     0000c53c  _USBBufferDataAvailable               
0     0000c548  _USBBufferSpaceAvailable              
0     0000c554  _USBBufferEventCallback               
0     0000c5c2  _USBStackModeSet                      
0     0000c5d8  _USB0DualModeIntHandler               
0     0000c612  _USBDualModeInit                      
0     0000c655  _USBDualModeTerm                      
0     0000c66e  _USBOTGModeTerm                       
0     0000c68a  _USBOTGModeInit                       
0     0000c6fa  _USBOTGPollRate                       
0     0000c702  _USB0OTGModeIntHandler                
0     0000c781  _OTGDeviceDisconnect                  
0     0000c78f  _USBOTGMain                           
0     0000c834  _USBDeviceConfig                      
0     0000c971  _USBDeviceConfigAlternate             
0     0000c9da  _IntMasterEnable                      
0     0000c9de  _IntMasterDisable                     
0     0000c9e2  _IntRegister                          
0     0000ca00  _IntUnregister                        
0     0000ca20  _IntEnable                            
0     0000ca47  _IntDisable                           
0     0000cae2  _Interrupt_enable                     
0     0000cb2c  _Interrupt_disable                    
0     0000cbd6  _USBDCDConfigDescGetSize              
0     0000cbef  _USBDCDConfigDescGetNum               
0     0000cc14  _USBDCDConfigDescGet                  
0     0000cc58  _USBDCDConfigGetNumAlternateInterfaces
0     0000cc7d  _USBDCDConfigGetInterface             
0     0000cc96  _USBDCDConfigGetInterfaceEndpoint     
0     0000cce5  _USBRingBufFull                       
0     0000ccfe  _USBRingBufEmpty                      
0     0000cd10  _USBRingBufFlush                      
0     0000cd23  _USBRingBufUsed                       
0     0000cd33  _USBRingBufFree                       
0     0000cd3e  _USBRingBufContigUsed                 
0     0000cd4d  _USBRingBufContigFree                 
0     0000cd67  _USBRingBufSize                       
0     0000cd6c  _USBRingBufReadOne                    
0     0000cd7f  _USBRingBufRead                       
0     0000cd98  _USBRingBufAdvanceRead                
0     0000cdae  _USBRingBufAdvanceWrite               
0     0000cdd2  _USBRingBufWriteOne                   
0     0000cde6  _USBRingBufWrite                      
0     0000cdfe  _USBRingBufInit                       
0     0000ce86  _USBLibDMAInit                        
0     0000cedf  _USBDescGetNum                        
0     0000cf05  _USBDescGet                           
0     0000cf30  _USBDescGetNumAlternateInterfaces     
0     0000cf7e  _USBDescGetInterface                  
0     0000cf98  _USBDescGetInterfaceEndpoint          
0     0000cfaa  _SysCtlPeripheralReset                
0     0000cfae  _SysCtlPeripheralEnable               
0     0000cfea  _SysCtlPeripheralDisable              
0     0000d026  _SysCtlPeripheralPresent              
0     0000d02b  _SysCtlDelay                          
0     0000d03c  _SysCtlClockGet                       
0     0000d044  _SysCtlUSBPLLEnable                   
0     0000d051  _SysCtlUSBPLLDisable                  
0     0000d056  FD$$ADD                               
0     0000d0f2  _USBUARTTXIntHandler                  
0     0000d13b  _USBUARTRXIntHandler                  
0     0000d188  _f28x_USB0DeviceIntHandler            
0     0000d1b9  _f28x_USB0HostIntHandler              
0     0000d1ea  _f28x_USB0DualModeIntHandler          
0     0000d21b  FD$$DIV                               
0     0000d2a6  FD$$MPY                               
0     0000d329  _InternalUSBTickInit                  
0     0000d34e  _InternalUSBTickReset                 
0     0000d352  _InternalUSBRegisterTickHandler       
0     0000d380  _InternalUSBStartOfFrameTick          
0     0000d3ab  _c_int00                              
0     0000d401  _USBGPIOEnable                        
0     0000d409  _USBGPIODisable                       
0     0000d411  _USBDelay                             
0     0000d453  C$$EXIT                               
0     0000d453  _abort                                
0     0000d455  _exit                                 
0     0000d47c  _InitPieCtrl                          
0     0000d49b  _EnableInterrupts                     
0     0000d4a4  _InitPieVectTable                     
0     0000d4ca  _copy_in                              
0     0000d4ee  _memcpy                               
0     0000d50c  FD$$TOUL                              
0     0000d527  __args_main                           
0     0000d540  UL$$TOFD                              
0     0000d569  _USB0DeviceIntHandler                 
0     0000d57b  FD$$SUB                               
0     0000d589  _IntDefaultHandler                    
0     0000d596  __register_unlock                     
0     0000d59a  __register_lock                       
0     0000d59e  __nop                                 
0     0000d59f  _DSP28x_usDelay                       
0     0000d5a3  __system_pre_init                     
0     0000d5a5  __system_post_cinit                   
0     0000d5a6  ___etext__                            
0     0000d5a6  etext                                 
1     00000400  __stack                               
1     00000800  __STACK_END                           
1     00000880  _DevEmuRegs                           
1     00000985  _SysPwrCtrlRegs                       
1     00000a80  _FlashRegs                            
1     00000ae0  _CsmRegs                              
1     00000b00  _AdcResult                            
1     00000c00  _CpuTimer0Regs                        
1     00000c08  _CpuTimer1Regs                        
1     00000c10  _CpuTimer2Regs                        
1     00000ce0  _PieCtrlRegs                          
1     00000d00  _EmuKey                               
1     00000d00  _PieVectTable                         
1     00000d01  _EmuBMode                             
1     00000d02  _Flash_CallbackPtr                    
1     00000d04  _Flash_CPUScaleFactor                 
1     00001000  _DmaRegs                              
1     00001400  _Cla1Regs                             
1     00004000  _Usb0Regs                             
1     00005000  _McbspaRegs                           
1     00006000  _ECanaRegs                            
1     00006040  _ECanaLAMRegs                         
1     00006080  _ECanaMOTSRegs                        
1     000060c0  _ECanaMOTORegs                        
1     00006100  _ECanaMboxes                          
1     00006400  _Comp1Regs                            
1     00006420  _Comp2Regs                            
1     00006440  _Comp3Regs                            
1     00006800  _EPwm1Regs                            
1     00006840  _EPwm2Regs                            
1     00006880  _EPwm3Regs                            
1     000068c0  _EPwm4Regs                            
1     00006900  _EPwm5Regs                            
1     00006940  _EPwm6Regs                            
1     00006980  _EPwm7Regs                            
1     000069c0  _EPwm8Regs                            
1     00006a00  _ECap1Regs                            
1     00006a20  _ECap2Regs                            
1     00006a40  _ECap3Regs                            
1     00006ac0  _HRCap1Regs                           
1     00006ae0  _HRCap2Regs                           
1     00006b00  _EQep1Regs                            
1     00006b40  _EQep2Regs                            
1     00006c80  _HRCap3Regs                           
1     00006ca0  _HRCap4Regs                           
1     00006f80  _GpioCtrlRegs                         
1     00006fc0  _GpioDataRegs                         
1     00006fe0  _GpioIntRegs                          
1     00007010  _SysCtrlRegs                          
1     00007040  _SpiaRegs                             
1     00007050  _SciaRegs                             
1     00007060  _NmiIntruptRegs                       
1     00007070  _XIntruptRegs                         
1     00007100  _AdcRegs                              
1     00007740  _SpibRegs                             
1     00007750  _ScibRegs                             
1     00007900  _I2caRegs                             
1     0000e000  _ebss_start                           
1     0000e38e  _g_psCDCSerSections                   
1     0000e394  _g_psCDCCompSerSections               
1     0000e39c  _g_pui8IADSerDescriptor               
1     0000e3a4  _g_pui8CDCSerDescriptor               
1     0000e3ad  _g_pui8CDCSerDeviceDescriptor         
1     0000e3c0  _g_pui8TxBufferWorkspace              
1     0000e3d8  _g_pui8RxBufferWorkspace              
1     0000e400  _g_sCDCDevice                         
1     0000e440  _g_pi8USBRxBuffer                     
1     0000e540  _g_pi8USBTxBuffer                     
1     0000e6cc  _g_bUSBTimerInitialized               
1     0000e6ce  _g_ui32CurrentUSBTick                 
1     0000e6d0  _g_ui32USBSOFCount                    
1     0000e6d2  _g_pfnTickHandlers                    
1     0000e6de  _g_pvTickInstance                     
1     0000e6eb  _g_iUSBMode                           
1     0000e6ec  _g_eOTGModeState                      
1     0000e6f0  _g_ui32PollRate                       
1     0000e6f2  _g_ui32WaitTicks                      
1     0000e6f4  ___TI_enable_exit_profile_output      
1     0000e6f6  ___TI_cleanup_ptr                     
1     0000e6f8  ___TI_dtors_ptr                       
1     0000e6fe  __lock                                
1     0000e700  _g_ppsDevInfo                         
1     0000e704  _g_psDCDInst                          
1     0000e7be  __unlock                              
1     0000e7c0  _PieVectTableInit                     
1     0000e90d  _g_pui8ConfigString                   
1     0000e976  _g_pui8ControlInterfaceString         
1     0000e9a2  _g_pui8ManufacturerString             
1     0000e9c6  _g_pui8CDCSerCommInterface            
1     0000e9e9  _g_pui8ProdectString                  
1     0000ea26  _g_sCDCHandlers                       
1     0000ea3e  _g_pui8CDCSerDataInterface            
1     0000ea55  _g_pui8SerialNumberString             
1     0000ea68  _g_sRxBuffer                          
1     0000ea7a  _g_sTxBuffer                          
1     0000ea9c  _g_pui8StringDescriptors              
1     0000eab4  _g_pui8LangDescriptor                 
1     0000eab8  _g_sCDCCompSerConfigHeader            
1     0000eabc  _g_sCDCSerCommInterfaceSection        
1     0000eac0  _g_sCDCSerConfigHeader                
1     0000eac4  _g_sCDCSerConfigSection               
1     0000eac8  _g_sCDCSerDataInterfaceSection        
1     0000eacc  _g_sIADSerConfigSection               
1     0000ead2  _g_pCDCCompSerConfigDescriptors       
1     0000ead4  _g_ppCDCSerConfigDescriptors          
1     003d7e80  _PartIdRegs                           
1     003f7ff8  _CsmPwl                               
abs   00000400  __STACK_SIZE                          
abs   000007c0  _ebss_size                            
abs   ffffffff  ___TI_pprof_out_hndl                  
abs   ffffffff  ___TI_prof_data_size                  
abs   ffffffff  ___TI_prof_data_start                 
abs   ffffffff  ___binit__                            
abs   ffffffff  ___c_args__                           
abs   ffffffff  ___pinit__                            
abs   ffffffff  binit                                 
abs   ffffffff  pinit                                 

[499 symbols]
